:07000300012501C101C1004C
:10000E00C2AFC28C5389F0438901758A03E4F58C23
:09001E00C2B9D2A9D28CD2AF22E2
:03000B00020027C9
:10002700C0E0C0F0C0D075D010C28C7403258AF52B
:100037008A858C8CD28C0527E52770020526AE268B
:10004700AF277C007D051207BFED4C70047F018050
:10005700027F00A202E4335F600EA2019280A20138
:0F0067009281A2019282B201D0D0D0F0D0E032CB
:1000760085262E85272FE52F2FFDE52E3EFCC3E591
:08008600279DE5269C40EF22B6
:10008E00E4FB2097100B7F0A7E00120076EBD394D0
:06009E001440EFD2002225
:0B00A400C280D281D282D284D283229B
:1000AF0085262E85272FE52F241FFFE4352EFEC32F
:1000BF00E5279FE5269E50307F0112062EA29282E1
:1000CF00918295B09450207F0212062EA2928291B7
:1000DF00B095829450117F0312062EA292829182C4
:0900EF0095B0945002D322C32203
:1000F80085262E85272FE52F241FFFE4352EFEC3E6
:10010800E5279FE5269E50307F0112062EA2928297
:10011800918295B09450207F0212062EA291B0923F
:100128008295829450117F0312062EA292829182A8
:0901380095B0945002D322C322B9
:10014100AB07751A00751B01E4FAEAC39B5012AEA6
:100151001AAF1B7C007D0A1207AB8E1A8F1B0A8017
:06016100E9AE1AAF1B22FB
:10016700E4F51885262E85272FE52F2464FFE4352F
:100177002EFEC3E5279FE5269E400302022B20970C
:1001870002C3221206D18F19EF24F6500F24F9600B
:100197000B24D1700302021C243070CD1206D1AD9E
:1001A70019ED3395E0FCEF6D7002EE6C60EE74288C
:1001B7002518F8A6190518C2837F027E001200765B
:1001C700D283E518B404A2752400752300752200B4
:1001D700752100E4F9C3E5186480F8E96480985054
:1001E70032AF24AE23AD22AC21120827E51814C381
:1001F70099FF120141742829F8E6FD3395E0FC12B6
:1002070007ABE4FCFD1208148F248E238D228C216A
:100217000980C2D322C3E518648094844003020195
:0602270070020170C32209
:10022D0085232C85242DE52DF534E52CFF3395E024
:10023D008F35753001E530C39525501CAF30120553
:10024D00C8EFB5340D0530AF301205C8EFB5350226
:10025D00D3220530053080DDC322E530C39525500E
:10026D002CAF301205C8EF6534701A0530AF30125F
:10027D0005C8EFB5350D0530AF301205C8EFB533F4
:0F028D0002D322053005300530053080CDC32265
:10029C0085232C85242DE52DF534E52CFF3395E0B5
:1002AC008F35AF25AD34120608EF60100525AF254C
:1002BC00AD35120608EF60040525D322C322C322F4
:1002CC0012022D40030203D6751800853019C3E5C0
:1002DC00199525E518940050580519E51970020573
:1002EC0018AF191205C88F340519E51970020518D5
:1002FC00AF191205C88F3574FD2519F51974FF3522
:10030C0018F518AF19AD34120608EF601A0519E587
:10031C001970020518AF19AD35120608EF60080503
:10032C0019E519700205180519E5197002051880F0
:10033C009D15251525D322C3E5199525E51894009F
:10034C0040030203CE0519E51970020518AF191206
:10035C0005C88F340519E51970020518AF19120577
:10036C00C88F350519E51970020518AF191205C8A3
:10037C008F3374FB2519F51974FF3518F518AF195F
:10038C00AD34120608EF602F0519E5197002051837
:10039C00AF19AD35120608EF601D0519E51970028D
:1003AC000518AF19AD33120608EF600B740225194E
:1003BC00F519E43518F5180519E519700205180238
:0C03CC00034374FD2525F525D322C32230
:1003D80085262E85272FE52F2432FFE4352EFEC3F0
:1003E800E5279FE5269E50541206D1EE70E8EF24CB
:1003F800F060261470E01206D1EF64114E60F7C267
:100408000212029C50D0C283D280C281D2827F075E
:100418007E00120076D283D3221206D1EF64104EEA
:1004280060F7C2021202CC50ADC283D280C282D21F
:0E043800817F077E00120076D283D322C3227A
:10044600D280C2837F057E00120076D2837F14128B
:100456000076E4F526F527C3E5279496E52694006D
:100466005018D20212016750EEE4F526F527120362
:0D047600D850E4E4F526F52780DDC202220F
:100483001200A412000E1200AF5037E4FF7D0112D8
:100493000608EF6015D280D281C282C2837F0A7EB2
:1004A30000120076D283D2828011D280C281C282AE
:1004B3007F0A7E00120076D281D2827F147E0012E0
:1004C30000761200F85017E4FF1205C88F251204B6
:1004D30046E4FFAD25120608EF60031200A420973F
:1004E30023D280C28120000312008E209716A2011E
:1004F30092837F087E00120076D2837F19120076E2
:10050300B20180DAC200C280D28112016750CFE407
:10051300FF1205C88F2512022D5016C284C2817F97
:100523000A7E00120076D2847F14120076D2818074
:10053300ADC282C2837F0A7E00120076D282D2834A
:03054300809C2277
:09054600C2A0D2A10000D2A02243
:0D054F00D2A0D2A10000C2A00000C2A122D3
:0E055C000000D2A10000A2A0E433FFC2A12241
:06056A00D2A012055C2284
:06057000C2A012055C228E
:10057600E4FED2A0FDEE25E0FE12055CEF60054329
:0E058600060180035306FE0DBD08EAAF0622F3
:10059400AE07E4FDEE3392A0EE25E0FE12055C0DFD
:0405A400BD08F1227B
:1005A800E4FC12054F7FA012059412056AEF70064D
:1005B8001205467F01220CBC80E81205467F002206
:1005C800AC0712054F7FA0120594120570AF0412F4
:1005D80005941205700000D2A10000D2A00000000E
:1005E800C2A0000000C2A10000007FA11205941261
:1005F8000570120576AE0712056A120546AF062287
:10060800AC07AB0512054F7FA0120594120570AF19
:1006180004120594120570AF0312059412057012A6
:0606280005461205A822A0
:10062E007590FFEF24FE600A14600A24027008C25F
:08063E009622C29322C2902211
:10064600EE60030206D0EF24FE60301460532402ED
:1006560060030206D0EC7072ED24FE600F14601188
:10066600146013240370637E007F01227E007F04E2
:10067600227E007F07227E007F1022EC704CED2444
:10068600FE600F1460111460132403703D7E007F1A
:1006960002227E007F05227E007F08227E007F00E8
:1006A60022AE04AF05EC7022EF24FE600F14601139
:1006B600146013240370137E007F03227E007F06DE
:0B06C600227E007F09227E007F1122AF
:1006D1007D057C007B017A00C3EB9404EA6480947D
:1006E100805036AF0312062E2094047C007D042036
:1006F10095047C007D032091047C007D01209204FF
:100701007C007D02ED64054C6008AF03AE02120669
:0E07110046220BEB70010A80BF7E007F402263
:0300000002071FD5
:0C071F00787FE4F6D8FD7581350207668E
:1007AB00EFF88DF0A4FFEDC5F0CEA42EFEEC88F093
:0407BB00A42EFE2248
:1007BF00BC000BBE0029EF8DF084FFADF022E4CC1E
:1007CF00F875F008EF2FFFEE33FEEC33FCEE9DECE7
:1007DF00984005FCEE9DFE0FD5F0E9E4CEFD22ED2D
:1007EF00F8F5F0EE8420D21CFEADF075F008EF2F77
:1007FF00FFED33FD4007985006D5F0F222C398FD68
:05080F000FD5F0EA2204
:10081400EF250BFFEE350AFEED3509FDEC3508FC3E
:0308240002084E79
:10082700E50C050C6010D0F0D0E0C008C009C00A84
:10083700C00BC0E0C0F08F0B8E0A8D098C0822AF69
:100847000BAE0AAD09AC08E50C146010D0F0D0E08F
:0F085700D00BD00AD009D008C0E0C0F0150C2299
:10072B00020483E493A3F8E493A34003F68001F25D
:10073B0008DFF48029E493A3F85407240CC8C333CF
:10074B00C4540F4420C8834004F456800146F6DF9E
:10075B00E4800B0102040810204080900003E47E2B
:10076B00019360BCA3FF543F30E509541FFEE49393
:10077B00A360010ECF54C025E060A840B8E493A35A
:10078B00FAE493A3F8E493A3C8C582C8CAC583CA85
:10079B00F0A3C8C582C8CAC583CADFE9DEE780BE3D
:01000A0000F5
:00000001FF
